:10000000370101002928A948730000008280135697
:10001000F50133A5A500518D1345150082804EB81A
:100020000111A2E4CAE052FC5AF862F46AF00565D4
:100030001309C0279304A0281304D029930BF02A96
:10004000194B9549930C702D130D402C130C902CCB
:100050008965930DB02E1566A566130505C62ACED3
:100060001385058C2ACC138505522ACA1305066A06
:100070002AC8138506482AC63DA83245419D2A9ABA
:100080005A899304A0281304D029194B130510335F
:100090009D225285A92A1305B033B12A13551A009F
:1000A000B92213056034812A13552A0089221305C9
:1000B00010359122692A4A853D2A26852D2A130565
:1000C000000235222285052A130530060D22294516
:1000D0003D225E850D22A52AAA8A112A29450522DC
:1000E00063ED6A016285012A5E8531228D22AA8A2A
:1000F000FD2829452922E3E759FF7245338AAA02E0
:100100002A9AE3853AF96685FD20338B59415A8551
:10011000F9286A85CD20252AAA84D1282945C52019
:1001200063779B006285C1286685F120CDB7A69ACA
:100130006245459D2A9A1145E36555F54A8B6E85C2
:100140005D28B384594126855D206A856D20012292
:100150002A847128294565201309303063F184020F
:10016000628551286E854128268551206A85612047
:10017000F9282A84AD2829455920E3E384FEA29A70
:100180005245419D2A9A1145E36C55EF4A85A520B9
:10019000B38459412685A1286A85B1284D282A842F
:1001A000B9202945A92863F784006285A9204A85DA
:1001B0009920CDB7A29A4245419D2A9A1145E36103
:1001C00055ED1309A0314A853D20B3845941268558
:1001D00039286A850D20A5282A841128294505205B
:1001E000E3FD84E8628501284A853120CDB7854842
:1001F0007300000082809148730000008280AD4847
:100200007300000082809308100873000000828051
:1002100093085008730000008280930870087300F0
:1002200000008280732510C08280732500C0828008
:10023000930860087300000082800589F322008023
:1002400093920248B3E2A2007390028082809548A4
:100250007300000082809308000873000000828011
:10026000A1487300000082809308300873000000EA
:100270008280930840087300000082800A0A0A53B3
:10028000657474696E67733A0A004261736520533E
:100290007461636B20436F756E743A20000A4D6180
:1002A0007820537461636B2053697A653A20000AA1
:1002B000537465656C2055706772616465733F0A9D
:1002C0005B302D355D203E2000496E76616C69649F
:1002D00020656E747279000A476F6C6420557067F0
:1002E00072616465733F0A5B302D000A4F62736967
:1002F0006469616E2055706772616465733F0A5B63
:10030000302D000A4469616D6F6E6420557067720C
:10031000616465733F0A5B302D000A4D6974687231
:10032000696C2055706772616465733F0A5B302D9C
:10033000000A3120736C6F743A20000A3220736C0B
:100340006F74733A20000A3420736C6F74733A2010
:10035000000A5072657373203020746F2072756EBE
:0803600020616761696E0A006B
:00000001FF
